:1000000012C02CC02BC02AC029C028C027C026C0BF
:1000100076C030C023C022C021C020C01FC01EC077
:100020001DC01CC01BC011241FBECFE5D4E0DEBF25
:10003000CDBF10E0A0E6B0E0EAE6F6E002C0059031
:100040000D92A036B107D9F710E0A0E6B0E001C0EC
:100050001D92A436B107E1F702D005C3D1CFDF93DB
:10006000CF93CDB7DEB733D2D9D280E090E0CF9135
:10007000DF9108951F920F920FB60F9211242F93C4
:100080003F934F935F936F937F938F939F93AF9320
:10009000BF93EF93FF93DF93CF93CDB7DEB78091FC
:1000A00062009091630018161906ACF4A9D185E39B
:1000B00090E025E330E0F901308122E02327FC01C4
:1000C0002083809162009091630001979093630078
:1000D0008093620001C078D0CF91DF91FF91EF91C2
:1000E000BF91AF919F918F917F916F915F914F9150
:1000F0003F912F910F900FBE0F901F9018951F9258
:100100000F920FB60F9211242F933F934F935F934B
:100110006F937F938F939F93AF93BF93EF93FF93CF
:10012000DF93CF93CDB7DEB780D1809160009091FF
:10013000610001969093610080936000CF91DF9100
:10014000FF91EF91BF91AF919F918F917F916F91AF
:100150005F914F913F912F910F900FBE0F901F9085
:100160001895DF93CF9300D0CDB7DEB79A838983FC
:1001700089819A81909363008093620088E390E084
:1001800028E330E0F90120812068FC0120831092EF
:1001900061001092600085E390E025E330E0F90112
:1001A00020812B7FFC01208340D12AD188E390E07D
:1001B00028E330E0F90120812F77FC0120830F90A4
:1001C0000F90CF91DF910895DF93CF9300D000D0AF
:1001D00000D0CDB7DEB785E390E025E330E0F9014C
:1001E00020812460FC01208383E590E0FC011082E3
:1001F0008CE490E0FC01808191819A8389838091D5
:1002000060009091610000249695879507949695DB
:1002100087950794982F802D9C01207C3F738981BE
:100220009A81892F992786958695822B932B9C837B
:100230008B838CE490E0FC01808191819C010024FF
:10024000369527950794369527950794322F202DBC
:1002500080E390E0FC01808182958695869583708D
:10026000882F90E0AC01507086E390E0FC01808123
:10027000882F90E087709070880F991F880F991FC2
:10028000482B592B80E390E0FC018081882F90E07F
:1002900080729070842B952B822B932B9E838D8361
:1002A00088E390E028E330E0F90120812068FC0138
:1002B00020838B819C812D813E81B901B5D185E35D
:1002C00090E025E330E0F90120812260FC012083E9
:1002D00026960FB6F894DEBF0FBECDBFCF91DF914B
:1002E0000895DF93CF9300D000D00F92CDB7DEB743
:1002F00019821C821B8237C08BE290E0FC01808156
:1003000088238CF50FD18D838981882F90E08130EF
:10031000910559F082309105C1F0009721F58D814A
:100320008A8389818F5F89831EC08D81882F90E0A9
:10033000982F88279C018B819C81822B932B9C83F7
:100340008B8389818F5F89830EC08D81882F90E098
:1003500090702B813C81822B932B9C838B83898192
:100360008F5F898300008981833030F28A81882FF2
:1003700090E08C36910539F08337910581F087360E
:10038000910539F010C081E3B3D08B819C81F2D00C
:100390000CC081E3ADD08B819C81E3DE06C081E39C
:1003A000A7D012DF02C080E3A3D00F900F900F9070
:1003B0000F900F90CF91DF910895DF93CF93CDB73A
:1003C000DEB781E390E022E0FC01208382E390E04D
:1003D000FC01108287E390E028EAFC01208388E397
:1003E00090E0FC01108284E390E027E0FC01208390
:1003F00085E390E022E0FC012083CF91DF91089516
:10040000DF93CF93CDB7DEB783E590E0FC01108298
:1004100082E590E021EBFC01208383E590E025E07C
:10042000FC012083CF91DF910895DF93CF93CDB767
:10043000DEB78FE490E0FC0110828EE490E026E0CD
:10044000FC0120838CE490E0FC01118210828AE49C
:1004500090E021E030E0FC013183208388E490E0EB
:1004600021E030E0FC0131832083CF91DF910895BA
:10047000DF93CF93CDB7DEB789E590E029E530E093
:10048000F90120812560FC012083CF91DF9108953F
:10049000DF93CF93CDB7DEB780E490E0FC0110820C
:1004A00089E290E021E0FC0120838AE290E028E1EB
:1004B000FC01208380E490E02EE8FC0120838DE2A3
:1004C00090E028E1FC012083CF91DF910895DF9334
:1004D000CF93CDB7DEB7F89481E590E02CEAFC012C
:1004E00020836BDFD5DFC4DF7894CF91DF9108954F
:1004F000DF93CF930F92CDB7DEB7898300008BE2F5
:1005000090E0FC018081882F90E0807290700097CD
:10051000B1F38CE290E02981FC0120830F90CF9110
:10052000DF910895DF93CF93CDB7DEB700008BE264
:1005300090E0FC0180818823D4F78CE290E0FC01FC
:100540008081CF91DF910895DF93CF930F92CDB744
:10055000DEB789838FE290E02981FC0120830000CF
:100560008EE290E0FC0180818823D4F70F90CF9138
:10057000DF910895DF93CF9300D0CDB7DEB79A8394
:10058000898387E390E027E330E0F901208124604C
:10059000FC01208388E390E028E330E0F90120812A
:1005A0002B7FFC012083FC0180818DE290E028E517
:1005B000FC012083FC01808185E390E025E330E0AD
:1005C000F90120812E7FFC01208380E0BDDF89813D
:1005D0009A81892F9927B8DF8981B6DF85E390E07A
:1005E00025E330E0F90120812160FC012083FC013A
:1005F00080818DE290E028E1FC01208387E390E098
:1006000027E330E0F90120812B7FFC012083FC01EE
:1006100080810F900F90CF91DF910895DF93CF935A
:10062000CDB7DEB75EDEFECFDF93CF9300D000D034
:10063000CDB7DEB79A8389837C836B8389819A8166
:10064000892F992755DF898153DF8B819C81892FE1
:1006500099274EDF8B814CDF0F900F900F900F90FA
:0A066000CF91DF910895F894FFCFC9
:00000001FF
